:1000000012C03FC018951895189518951895189511
:100010001895189518951895189518951895189578
:100020001895189518958FED8DBFC0ECE0EC4E2E0D
:10003000DD275D2EEEE7F0E0A0E6B0E0A89584B7FE
:10004000082E877F84BF88E1992781BD91BD8827CD
:100050008D933197E9F766248FE087BB80E088BBFA
:100060008BE781BB84E082BB78948BB780648BBFC5
:1000700081E787BB8EE088BB85B7816285BF8895A5
:10008000F7CFF894E2E3F0E0AEE691E0AFD3009171
:100090006E000E3C08F004C085B7816285BF88956C
:1000A00080916F00806880936F0080E080936A0089
:1000B00080E080936900ACE66ED3A1E66ED380E069
:1000C00080936500ACE6FCD288E787BB87E088BBFD
:1000D00081E090E051D381E080936000A6E30C9131
:1000E00001FB81E00EF480E08F93A6E30C9100FB0E
:1000F00081E00EF480E09F918923882309F401C0F8
:1001000017D182E080936000A6E30C9101FB81E0AF
:100110000EF480E08F93A6E30C9100FB81E00EF0DB
:1001200080E09F918923882309F401C001D183E0F5
:1001300080936000A6E30C9101FB81E00EF080E06B
:100140008F93A6E30C9100FB81E00EF480E09F9179
:100150008923882309F401C0EBD084E787BB8BE0B7
:1001600088BB81E090E008D384E080936000A6E340
:100170000C9101FB81E00EF480E08F93A6E30C91DB
:1001800000FB81E00EF480E09F918923882309F42D
:1001900001C0CED085E080936000A6E30C9101FB06
:1001A00081E00EF480E08F93A6E30C9100FB81E0E8
:1001B0000EF080E09F918923882309F401C0B8D014
:1001C00086E080936000A6E30C9101FB81E00EF0D5
:1001D00080E08F93A6E30C9100FB81E00EF480E0B9
:1001E0009F918923882309F401C0A2D082E787BBAD
:1001F0008DE088BB81E090E0BFD287E08093600013
:10020000A6E30C9102FB81E00EF080E08F93A6E361
:100210000C9100FB81E00EF480E09F9189238823FC
:1002200009F401C085D088E080936000A6E30C91BA
:1002300002FB81E00EF480E08F93A6E30C9100FBBB
:1002400081E00EF080E09F918923882309F401C0AA
:100250006FD089E080936000A6E30C9102FB81E0FF
:100260000EF480E08F93A6E30C9100FB81E00EF486
:1002700080E09F918923882309F401C059D081E748
:1002800087BB8EE088BB81E090E076D28BE08093E4
:100290006000A6E30C9102FB81E00EF080E08F93FA
:1002A000A6E30C9101FB81E00EF480E09F9189238D
:1002B000882309F401C03CD08AE080936000A6E363
:1002C0000C9102FB81E00EF480E08F93A6E30C9189
:1002D00001FB81E00EF480E09F918923882309F4DB
:1002E00001C026D08CE080936000A6E30C9102FB55
:1002F00081E00EF480E08F93A6E30C9101FB81E096
:100300000EF080E09F918923882309F401C010D06A
:1003100081E090E031D2ACE60D911C91083E53E0B3
:10032000150710F009F001C0CDCE78941895089506
:10033000AFE68C9187FB81E00EF080E08F93009117
:1003400060000A3081E009F080E09F9189238823D2
:1003500009F409C08CEE93E1ACE68D939C93E1E047
:10036000F0E0B5D10895ACE616D2939A84E690E019
:1003700003D2939886E990E0FFD1BF98AFE69C91B5
:1003800096FF04C0B7990EC09F7B9C93B79B0AC091
:1003900088E29F939927F0D19F91B79B03C0906407
:1003A0009C934FD1AFE68C9187FB81E00EF080E00B
:1003B0008F93009160000B3081E009F080E09F9105
:1003C0008923882309F409C080916F008F77809377
:1003D0006F0084E690E0D0D108950091690001306B
:1003E00009F00DC08091600080936A00A9E68C91AD
:1003F0008F5F8C9380E080936500CBD0089500914F
:100400006900023009F001C04DC00091690003305D
:1004100009F001C066C0009160000B3009F008C00F
:10042000A9E68C918F5F8C9380E08093650008959E
:10043000009160000C3009F034C046E65BE260E0F9
:1004400070E0A1E60D911D912D913C91B1D109F083
:1004500001C08EC081E08093660000916600083084
:1004600010F009F01DC0E6E6F0E0A190EEEFFFEF1E
:10047000AA0CBB1CAA0CBB1CEA0DFB1DA4E194E05A
:10048000B5D1A1E60D911D912D913C9191D109F02D
:1004900001C0A6C0A6E68C918F5F8C9308F4DDCFD7
:1004A00067C03AC0009160000C3009F019C0E2E06A
:1004B000F0E0A4E194E09AD1A1E60D911D912D9177
:1004C0003C9176D109F401C053C063D0A1E665D157
:1004D00080E080936500A9E68C918F5F8C930895EE
:1004E0001BC0009160000C3009F016C0EAE6F0E095
:1004F000A190EEEFFFEFAA0CBB1CAA0CBB1CEA0DEF
:10050000FB1DA1E694E07BE760D143D08CEE93E144
:10051000ACE68D939C930895A5E68C918F5F8C93A8
:1005200000916500063010F009F001C001C020C044
:10053000A1E60D911D912D913C914AE050E060E0C3
:1005400070E0CBD0A1E60D931D932D933D93A1E6D2
:100550000D911D912D913C91A0E64C915527662758
:10056000772721D1A1E60D931D932D933D930895F7
:10057000ABE68C918F5F8C9389E0809367008FE569
:10058000809368000ED08CEE93E1ACE68D939C9343
:10059000089582E08093670088EC8093680001D022
:1005A000089584E690E0E8D081E080936600409171
:1005B000670000916600041710F009F010C0939ACC
:1005C000A8E68C919927D8D09398A8E68C91992782
:1005D000D3D0A6E68C918F5F8C9308F4E8CF089572
:1005E00080916E00815080936E00E2E3F0E0AEE611
:1005F00091E07BE7EAD080E080936B00A1E6CDD06C
:10060000C8DFE2E2F0E0A8E6EED000916800093031
:1006100010F009F001C003C089E08093680084EF06
:1006200091E0AAD0949AA8E6EC91FF2750D0949834
:10063000E1E0F0E04CD08CEE93E1ACE68D939C933E
:100640000895E4E0F0E043D0B79901C030C08FEFE7
:100650008093680081E080936600009166000E320E
:1006600010F009F00DC0A6E6EC91FF27A8E691E096
:100670007BE7ABD0A6E68C918F5F8C9308F4EDCF2F
:10068000E6E2F0E002ED14E020E030E0A0E1BB277C
:1006900094E07BE79AD0E2E2F0E001E010E020E0B5
:1006A00030E0A0E1BB2794E07BE78FD072DFB79BFF
:1006B00001C0FDCF8CEE93E1ACE68D939C93089541
:1006C000ED91FC91EF5FFF4FFC93EE93089588EE60
:1006D00093E052D03197D9F7089522D006D000FC8C
:1006E00001D0089528D030D00895842F952FA62FBB
:1006F000B72F4427552766277727F1E2889409C04A
:1007000020F4480F591F6A1F7B1F769567955795F0
:1007100047953795279517950795FA9589F7089581
:100720000024E89477FF02C006D0689400F809D04E
:1007300010F80124089512D04F5F5F4F6F4F7F4F25
:100740000895E89437FF0895009510952095309509
:100750000F5F1F4F2F4F3F4F68940895409550955E
:100760006095709508953197F1F70895689462F84F
:100770000895E89462F80895EF93FF93EE27E82B2D
:10078000E92B31F0EAEFF0E03197F1F70197D1F77B
:10079000FF91EF91089582E001C084E099279D9335
:1007A0008A95E9F70895040F151F261F371F08952E
:1007B00004171507260737070895E199FECFEEBB0A
:1007C0003196089591E001C092E07B3751F47FB7F4
:1007D000F894F3DF8D918DBBE29AE19A9A95C9F76F
:1007E0007FBF7727089591E001C092E0E6DFE09AAD
:0A07F0008DB38D939A95D1F708950B
:00000001FF
